:020000040000FA
:10000000F2EF03F01200FFFF04EF04F01200FFFF15
:10001000FFFFFFFFFFFFFFFF0CEF04F01200FFFFE9
:10002000FFFFFFFFFFFFFFFFFFFF0100FC070000D6
:100030006C0000000400000000017C6B1E0E716E5D
:100040000401400E096F200E0A6F040E0B6F880E1C
:10005000086F0401200E0E6F040E0F6F400E0C6F20
:100060001200550EA76EAA0EA76EA68212000401FA
:10007000226B010E236F120000017A6B04012151E3
:1000800000017A5D20E27AC000F0016A026A040190
:1000900022510024F36E23510120F46E24510220DA
:1000A000F86EF4CFF7FFF3CFF6FF0800F5CF7BF043
:1000B00000017A51EA6A250FE96E040EEA227BC03C
:1000C000EFFF7A2BDBD7F86A1200F00E040122173B
:1000D000840EA66E00017A6B0401215100017A5D45
:1000E00026E27A51EA6A250FE96E040EEA22EFCF82
:1000F00003F07AC000F0016A026A04012251002470
:10010000F36E23510120F46E24510220F86EF4CFD7
:10011000F7FFF3CFF6FF03C0F5FF0C000F0E000151
:100120007A150F0801E19DDF00017A2BD5D7120067
:10013000940EA66E00017A6B0401215100017A5DD4
:100140001EE27A51006E016A060ED8900036013622
:10015000E804FBE1026A01BE0268040122510024A6
:10016000F36E23510120F46E24510220F86EF4CF77
:10017000F7FFF3CFF6FF75DF00017A2BDDD7F86AC2
:100180001200A66A00017A6B0401215100017A5D18
:1001900010E20401225100017A25A96EA6807A514D
:1001A000EA6A250FE96E040EEA22A8CFEFFF7A2B48
:1001B000EBD7120000017A6B0401215100017A5D36
:1001C00015E20401225100017A25A96E7A51EA6AEA
:1001D000250FE96E040EEA22EF50A86E040EA66EFB
:1001E00040DFA6B2FED700017A2BE6D71200C40E7C
:1001F000A66E00017A6B0401215100017A5D21E2B3
:100200007A51EA6A250FE96E040EEA22EFCF03F075
:100210007AC000F0016A026A040122510024F36EE0
:1002200023510120F46E24510220F86EF4CFF7FF21
:10023000F3CFF6FF03C0F5FF0C0013DF00017A2BAC
:10024000DAD7F86A1200060E00017F5D03E36D50F5
:10025000020B01E074D000017C0511E104010CBF28
:100260000DD00401400E096F400E0401081704016F
:10027000087D880E0401081300017C6B60D0040126
:1002800008BF5DD000017A6B04012051320A45E0BD
:10029000CD0A34E0F80A2DE0020A26E0010A1FE048
:1002A000070A18E0010A11E0030A0AE0070A08E059
:1002B000060A01E033D0DBDE0001040E7A6F2FD096
:1002C000DBDE050E00017A272AD0FFDE0001010ED9
:1002D0007A6F25D02DDF0001010E7A6F20D051DF1B
:1002E000050E00017A271BD065DF0001010E7A6F31
:1002F00016D07DDF0001010E7A6F11D06D960001DE
:100300007D6B7E6B00017D07000E7E5B00017D51E1
:100310007E1101E0F7D7FF0002D001D000D000012C
:10032000010E7C6F00017A510AE07AC00DF4400E94
:1003300004010C1704010C7D880E04010C1312003B
:100340006C5002E0000E01D0010E00090BE0040128
:1003500000513C0BE842E8420D0802E1BBEF01F01E
:10036000C4EF01F06C5002E0000E01D0010E040950
:1003700001E019D812000001606B616B666B676B5E
:1003800099EC02F046EF02F0020E0001605D09E117
:100390005CD8040100BD02D0C80E01D0880E006FE9
:1003A00012008BEF02F0040E00017F5D09E112C420
:1003B0006EFF6E50000802E2050E01D0030E7F6F43
:1003C0000001600509E10AD8040104BD02D0C80E8D
:1003D00001D0880E046F12008BEF02F00001080EAE
:1003E000665D000E675903E266C069F002D0080E30
:1003F000696F69C005F46951006E016A0050665F5B
:100400000150675B180E646F040E656F69511CE044
:10041000000180A307D062C0F6FF63C0F7FF0800A9
:10042000F55005D062C0E9FF63C0EAFFEF5064C039
:10043000E9FF65C0EAFFEF6E0001622B000E632347
:10044000642B65236907E2D7120001C46AF000013A
:100450006A516625666F000E6721676F180E626F1E
:10046000040E636F6A5111E062C0E9FF63C0EAFFE6
:10047000EF5064C0E9FF65C0EAFFEF6E642B000E29
:100480006523622B63236A07EDD7120000016151D7
:100490000BE10401080E016F100E026F040E036FD2
:1004A000840E006F040123D0040110AF22D000019C
:1004B00066510401165D000167510401175904E2F9
:1004C00016C466F017C467F089DF0001010E606F83
:1004D0000401080E016F100E026F040E036F800EF0
:1004E000006F0401180E066F040E076FC80E046F2C
:1004F00010D00001020E606F0401056BC80E046F7E
:100500000401080E016F180E026F040E036FC80E6F
:10051000006F6D9812000001606B0401080E016FFE
:10052000100E026F040E036F880E006F0401046B3F
:10053000120004011051600BE842E842E842E84230
:10054000E842000901E012001151080A39E0010AED
:1005500035E00F0A0AE0030A01E012000001010E73
:10056000616F0001040E7F6F12000001010E616FC8
:100570000401130507E10001AE0E626F070E636F01
:10058000120E13D0020E135D07E10001C00E626F60
:10059000070E636F200E09D0030E135D0AE1000100
:1005A000E00E626F070E636F040E0001666F676BEB
:1005B00002D00001616B000180831200EEEF02F0B7
:1005C0000001010E616F0001810E626F000E636F0A
:1005D000000180930001010E666F12000001010E00
:1005E000616F12C481F00401125104E10001050E93
:1005F0007F6F12000001060E7F6F1CEF00F0080EE7
:100600006D6E6DBAFED7686A110E696E0001020E3A
:100610007F6F12006850040B06E06950040B03E082
:100620006D92699468946850010B04E06950010B65
:1006300001E027D86850100B09E06950100B06E064
:10064000698468986D82A08A0300A19A6850200B83
:1006500009E06950200B06E070A003D08BEC02F09B
:100660007090689A030E00017F5D01E209D0685026
:10067000080B06E06950080B03E0A0EC01F0689657
:100680001200686A7B0E696E6E6A160E706E68A63E
:1006900002D06896FCD76D988BEC02F00001816B5C
:1006A0000001030E7F6F12002A0EF66E000EF76E29
:1006B000000EF86E00010900F550756F0900F55045
:1006C000766F03E1756701D03DD00900F550706F7A
:1006D0000900F550716F0900F550726F09000900AB
:1006E000F550E96E0900F550EA6E090009000900AD
:1006F000F550736F0900F550746F09000900F6CFCB
:1007000077F0F7CF78F0F8CF79F070C0F6FF71C0CE
:10071000F7FF72C0F8FF0001735302E1745307E062
:100720000900F550EE6E7307F8E27407F9D777C049
:10073000F6FF78C0F7FF79C0F8FF00017507000EDB
:10074000765BBFD71200C1CF83F00F0EC1127F0EB0
:10075000F16E0001846B938494908280CF6ACE6A9C
:100760009E90310ECD6E81A404D083C0C1FF00EFF6
:1007700004F0140E6F6EFFEC02F00AEC03F023ECB1
:1007800001F09EA012D09E900001842B0F0E00015C
:10079000845D0BE30001846B8250010B010A010BA5
:1007A000F36EFE0E8214F310826EE7D71200120170
:1007B000000200000008D8040B0000000000000147
:1007C000090220000101008032090400000200003B
:1007D00000000705010240000007058102400000FB
:1007E0000403090413EE00F023EE00F0F86A059C00
:1007F00054EC03F0A3EC03F0FDD712006B695DEA43
:100800000BEF16F01200FFFF40EF14F01200FFFF95
:10081000FFFFFFFFFFFFFFFFB6EF14F01200FFFF27
:10082000FFFFFFFFFFFFFFFFFFFF0100422C000063
:10083000600000007C000000E5DB0001010EF66FA7
:10084000F76FF86F330EF06FE66A43DBE552000195
:10085000F169F2691200D9CFE6FFE1CFD9FF070EA7
:10086000E126060E0001F95D03E36D50020B0AE07C
:100870000001F107000EF25B0001F151F21101E1FC
:10088000FF007ED10001F651040A01E155D1070AAB
:1008900001E11CD1010A1DE0030A01E06DD1EFC0A6
:1008A000E6FF010EE66E3DDBE552E552010EE66E17
:1008B000F30EE66E000EE66EF6EC0FF0E552E55232
:1008C000E552000905E0F3C0F4F00001020EF66FF6
:1008D00057D10201D25101E0F8D0FF0E0001F45DC2
:1008E00007E131DB000903E00001010EF66FEDD0F6
:1008F000FE0E0001F45D07E137DB000903E00001B3
:10090000010EF66FE2D0800E0001F45D06E10001F9
:10091000F56B0001030EF66FD8D0810E0001F45D77
:1009200031E1EFC0E6FFE66AFCDAE552E552000E7F
:10093000E66E020EE66E000EE66E010EE66E9BECB3
:1009400009F0E552E552E552E552E76E060EE7CFB3
:10095000DBFF060EDB040BE1EFC0E6FF010EE66EE7
:10096000E0DAE552E5520001040EF66F0AD0EFC05E
:10097000E6FF010EE66ED5DAE552E5520001010E02
:10098000F66FA3D0820E0001F45D11E10001010EAB
:10099000EF6FEFC0E6FF020EE66EC3DAE552E552F6
:1009A0001DDB000903E00001010EF66F8ED0830EFF
:1009B0000001F45D10E10001EF6BEFC0E6FF020EF5
:1009C000E66EAFDAE552E55209DB000903E000010B
:1009D000010EF66F7AD0800E0001F45D55E2030E31
:1009E0000001F415E76E010EE7CFDBFF0C0E0001EE
:1009F000F415E840E8403F0BE76E020EE7CFDBFF5F
:100A0000020EDB50030805E1020EF36E020EF3CF77
:100A1000DBFF300E0001F415E8380F0B010FE76E15
:100A2000030EE7CFDBFF030EDB50030805E1040EE6
:100A3000F36E030EF3CFDBFF060E146E400E0001C3
:100A4000F41514C0E7FFE75204E0E8427F0BE70625
:100A5000FCE1E76E040EE7CFDBFF040EDBCFE6FF21
:100A6000020EDBCFE6FF010EDBCFE6FF030EDBCF8E
:100A7000E6FFEBD8E552E552E552E552000903E006
:100A80000001010EF66F21D0DF6A0E0EDF5C1AE264
:100A9000DF50EA6ACE0FE96E000EEA22EF50000145
:100AA000F45D0EE1EFC0E6FFE66A3BDAE552E5529F
:100AB000DFCFE6FF150EE66E18EC0CF0E552E552BE
:100AC000DF2AE3D70001010EF66F5AD0EFC0E6FF30
:100AD000E66A27DAE552E552000EE66E020EE66E91
:100AE000000EE66E010EE66E17DBE552E552E552AA
:100AF000E552E76E050EE7CFDBFF050EDB501BE08E
:100B0000050EDB040EE1000EE66E020EE66E000E30
:100B1000E66E010EE66E6BEC0DF0E552E552E55225
:100B2000E5520001010EF66FEFC0E6FF010EE66E22
:100B3000F8D9E552E55224D0EFC0E6FFE66AF1D9D4
:100B4000E552E552000EE66E020EE66E000EE66E0F
:100B5000010EE66E6CDBE552E552E552E552000906
:100B60000AE00001010EF66FEFC0E6FF010EE66E2F
:100B7000D8D9E552E55204D00001010EF66F00D03D
:100B8000070EE15C02E2E16AE552E16EE552E7CF71
:100B9000D9FF120005EC0BF0EFC0E6FFE66AC1D901
:100BA000E552E552F0C081FF140EE66E93DAE5528D
:100BB000FE0EDB500B0DF3CFECF00001F35028ECF0
:100BC0000BF0EECFEDF0EDCFEEF0F32828EC0BF0CC
:100BD000EECFE2F0EDCFE3F0020EF32428EC0BF0C1
:100BE000EECFE4F0EDCFE5F0030EEC27DE6BDF6B2C
:100BF000E06BE16BDD6BF28C96EC0BF0BD6A050EE1
:100C0000BD6E9E6AF28EDDA5FED7F29E330E816E1A
:100C1000DDB303D070EC0BF016D0EA51E65DEB517A
:100C2000E7590BE2E851E91104E0E807000EE95B3F
:100C300004D070EC0BF0EA6BEB6BEA51E65DE66F0B
:100C4000EB51E759E76F0AEF0BF005EC0BF0410EA3
:100C5000E1263B0EDB6A360EDB6A030EF36E370EBF
:100C6000F3CFDBFF020EF36E380EF3CFDBFF010E86
:100C7000F36E390EF3CFDBFFFD0EDBA003D03C0E8D
:100C8000DB6A05D0030EF36E3C0EF3CFDBFFFD0EE7
:100C9000DBA202D0040E01D0030EF36E3D0EF3CFA3
:100CA000DBFF0001F751060A01E1F0D0030A01E180
:100CB000DED0010A01E1C5D0070A01E1B5D0010A81
:100CC00070E0030A01E0E9D00201C86B180EC85DAC
:100CD00006E2F9EC0AF0EE6AED6AC82BF7D7400E8F
:100CE000DB6AFE0EDB50F36E400ED7EC0BF054E2E5
:100CF0003C0EDB50E76E3E0EE7CFDBFF3D0EDB50D8
:100D0000F36E3E0ED7EC0BF044E2D950360F146E62
:100D1000DACF15F03E0EDB500F011424E96E000E01
:100D2000DA20EA6EEF50E66EC5D8E552FC0EDB50D5
:100D3000020819E13F0EDB6ADB50010827E33F0E92
:100D4000DBCFE6FFC6D8E552D1EC0AF0D8A002D03E
:100D5000CBEC0BF0D9CF14F0DACF15F0B4EC0BF0EC
:100D60003F0EDB2AE9D73F0EDB6AFC0EDB5003089F
:100D700005E0FC0EDBCFE6FFACD8E552D1EC0AF083
:100D8000D8A002D0CBEC0BF0B4EC0BF03E0EDB2A7B
:100D9000B5D7400EDB2AA5D70201C86B180EC96F64
:100DA00072D0FD0EDBA00CD0520EF36E300EF3CFDE
:100DB000DBFF470EF36E310EF3CFDBFF420E0BD09D
:100DC0005F0EF36E300EF3CFDBFF5F0EF36E310E6E
:100DD000F3CFDBFF5F0EF36E320EF3CFDBFFFD0EC2
:100DE000DBA202D0570E01D05F0EF36E330EF3CFAD
:100DF000DBFFFC0EC0EC0BF0340EE7CFDBFF3A0E4E
:100E0000F36E350EF3CFDBFF0201D2510DE102018B
:100E1000D950300FD36FDACFD4F20201060ED76F5C
:100E200013EC0BF00001F72B0201D25138E1020163
:100E30003B0ED36F2C0ED46F0201060E59EC0BF053
:100E400022D0D9CF14F0DACF15F00201D2DBEECFE9
:100E5000E6FFEFCFE6FFFBD8E552E552000902E0DE
:100E60000201C82B0201C951C85D19E30CD002016F
:100E7000D25115E10201380ED36F2C0ED46F02014E
:100E8000020E59EC0BF00001F72B09D0010EF76FA1
:100E9000F36E3B0EF3CFDBFF02D0010EF76F3B0E7C
:100EA000DB50146E410EE15C02E2E16AE552E16E54
:100EB0001450B0D3AADBFE0EDBA003D00001F08DEE
:100EC00002D00001F09DDBA202D0F08F01D0F09F94
:100ED000A1D39BDB040EE126D9CFE6FFDACFE6FFF4
:100EE000EED9E552E552020EDB50E76E030EE7CF76
:100EF000DBFFFE0EDB5004E1030EDB50020803E0D3
:100F0000030EDB5004E10001F081F09903D00001F1
:100F1000F091F089040EE15C02E2E16AE552E16ED3
:100F200079D373DBFE0EDB50020803E0FE0EDBCF4D
:100F3000CAF2FD0EDB5003E00201CA5102E18290C9
:100F400001D0828067D3BCEC0BF00201D25109E1E1
:100F50000201300ED36F2C0ED46F0201070EA9DBF5
:100F6000DF6EDF50E55256D350DB0C0EE126DF6A10
:100F7000D950090FE66E000EDA20E66EA0D9E552D0
:100F8000E552DE52760EDD6E090EC0EC0BF0020E5D
:100F9000E7CFDBFF2E0EF36E030EF3CFDBFF0A0E5F
:100FA000A6DB2E0EF36E050EF3CFDBFF0B0EA4DBDC
:100FB0000D0EC6DB0A0EBFDB0201D25105E180DB5C
:100FC000080ED76F30DBDF6EDF50146E0C0EE15C65
:100FD00002E2E16AE552E16E14501CD3CDDB02015E
:100FE000D2510DE102012E0ED36F2C0ED46F0201EF
:100FF000010ED76F0201D86F0201D26FDF6EDF5092
:10100000E55208D3806A826A330E816E92680C0EB4
:10101000936EFE0E946ED06A400EF26E800EF16EEC
:10102000050E9D6ECD6ABD6ECA6E0F0EBA6E0001C2
:10103000010EEF6F1200110ECB6E090EBB6E040E87
:10104000CA6E0F0EBA6E0001DC6B94921200DDDAEC
:10105000090EE126DF6AFE0EDB50E76E070EE7CFD2
:10106000DBFF640EC9DA09C0DBFF8ADB010EE7CFC4
:10107000DBFF640EC1DADDDA020E86DB81DB030EF4
:10108000E7CFDBFFFD0EDBCF14F0FE0EDBCF15F05C
:101090000001156A070E14C0DBFF640EADDA09C04B
:1010A000DBFF25DB640EA8DAC4DA050E6DDB24DB7A
:1010B0000201D25105E104DB060ED76FB4DADF6E10
:1010C000DF50146E090EE15C02E2E16AE552E16E66
:1010D0001450A0D29ADA020EE126DF6AFE0EDB502F
:1010E000DF5C13E2010EDB6ADF50146E156AD890E4
:1010F000155004E6FA0E145C000E155804E2DF2ABF
:10110000DF06DF2AF1D7DF2AE9D7020EE15C02E22F
:10111000E16AE552E16E7ED22FDB0001F55107E175
:10112000010EF56F0201CB6BCC6BCD6BCE6B010E5C
:10113000E66EF30EE66E000EE66EF6EC0FF0E5528C
:10114000E552E552000966E00201CD6BCE6BC80E98
:10115000CB5D000ECC590BE2FD0EDB50CB250F0111
:10116000E96EFE0EDB500201CC210F010FD0CBC285
:1011700014F0CCC215F0C80E145E000E155AFB0E0A
:10118000DB501424E96EFC0EDB501520EA6EF3C030
:10119000EFFF0201CB2B000ECC23900ECB5D010E96
:1011A000CC5902E3020E3FD0080ECB5D000ECC59A5
:1011B0003BE302DB500803E0FFDA600806E10C0EB7
:1011C000CB5D000ECC5930E323D0040EE3D9EFCF32
:1011D00018F0060EDFD9EF501824166E176A000EAD
:1011E0001722040E086E096A16C00DF017C00EF023
:1011F000B0EC15F006C014F007C015F0080E142668
:10120000000E152202011450CB5D1550CC590CE391
:10121000010E09D00201CD2B000ECE23CD1D04E11D
:10122000CE1D02E1020EDF6EDF50E552F3D1A4DAEB
:101230000001F851030A2EE0010A17E0030A3AE11F
:10124000040E086E096A04C10DF005C10EF0B0EC81
:1012500015F006C0CFF207C0D0F2080E0201CF276A
:10126000000ED0230001F82B27D00201D25112E149
:101270000201C80ED880CF55000ED05504E341DAE4
:1012800090DAF86F07D03DDA0201C80ED76FCBD9DC
:101290000001F82B0201D2510FE10201C80ECF5F0D
:1012A000000ED05BFB0EDBCFD3F2FC0EDBCFD4F213
:1012B00078DA01D0010EF86FDF50E552ABD1A5D935
:1012C000030EE126DF6A010EDB6A200EF36E020ECA
:1012D000F3CFDBFFD7D90800F550E66E36DAE552DA
:1012E000E750EF6ECFD9F62A13DA010E69DAEF6E06
:1012F000C9D9F6260DDA020E63DAEF6E26DAEF5060
:10130000FF0803E122DA010EEF6E56DAFF0803E16F
:10131000010E40D9EF6A020E3DD9EF50FF0804E1FB
:10132000020E38D9020EEF6E030EE15C02E2E16AB2
:10133000E552E16E6FD169D90E0EE126040EDB6A2B
:10134000070EDB6A050EDB68040EF5D9DE68DD6882
:10135000020EDB6A030EDB6A0B0EDB6A0C0EDB6A25
:101360000D0EDB6AF2D9EE6AED6A020E13D96D0E2C
:10137000EE6EED6A040E0ED9EE6AED6A060E0AD91B
:10138000EE6AED6A010EE66EA4DDE552F0C081FF63
:10139000BD6A050EBD6ECAD9010ECA6ECC6A4F0E6B
:1013A000CB6E050ECA6E9E6A070EDB5001E0D6D0EA
:1013B0009EB215D09EA4FCD79EA003D0DE68DD6847
:1013C0000AD0BF50166E176A176E166ABE50A7D99C
:1013D00014C0DEFFDD6EAAD99E949E90E9D79E923E
:1013E000CF50166E176A176E166ACE5098D9020E35
:1013F00014C0DBFF030E15C0DBFF9EA004D0020E5D
:10140000DB68030EDB68DECF14F0DDCF15F0780E5D
:10141000145C020E155811E2020EDBCF16F0030E1B
:10142000DBCF17F0780E165C020E175806E2010E9D
:10143000F36E060EF3CFDBFF02D0060EDB6A050E5D
:10144000DB50FF081DE1060EDB0401E179D0D95025
:101450000B0FE96EDACFEAFFEE2A000EEE22EE2243
:10146000D9500B0FE96EDACFEAFFE868EE189CE17D
:10147000E868EE1899E1050EEE1896E1020E5CD0D0
:10148000050EDB50F36E060EDB50F35C1BE1090E1C
:10149000DB2A0A0E01E3DB2AD950090FE96EDACF05
:1014A000EAFFFF0EEE1801E07FD7080EED1801E00D
:1014B0007BD7010E45D9B2D802E2EDD801D0D2D8FF
:1014C00007D972D7ABD802E2E6D801D0CBD800D981
:1014D000080EDB50146E156AC70E14182FE1155054
:1014E0002DE19CD824E3FB0EDBCF16F0FC0EDBCF06
:1014F00017F0080EDB509C0F020D1650F324E96E16
:101500001750F420EA6EEECF14F0EFCF15F0000E76
:10151000145C020E15580BE2020E146E080EDBCF9F
:10152000E7FF1450E75E080EE7CFDBFFDAD776D887
:1015300002E2C70E00D9010E03D936D7080EDB2A06
:10154000010EF36E090EF3CFDBFF0A0EDB6A060E07
:10155000DB50E76E050EE7CFDBFF26D7080EDB502A
:10156000FD0FFE0BE842E66E040E2AD9EE6EED6A20
:10157000330E816E070EDB50E76E040EE7CFDBFF04
:10158000DB50146E0E0EE15C02E2E16AE552E16EA0
:10159000145040D0E76ED9D8E750E926000EEA2271
:1015A0001200FB0EDBCFE6FFFE0EDB04E552E72464
:1015B000E66ECAEC05F0E5523F0EDB500C0DF3CFA2
:1015C00014F03E0EDB50030DF35014240201C86FDB
:1015D000020EC825C1D80001E051EE26E151ED22EE
:1015E0000201C829B9D80001E651EE26E751ED22E3
:1015F0001200C851ACEF0BF0146E0E6E070EDBCF6D
:1016000009F0FDEC15F0080E1200D9CFE6FFE1CF8E
:10161000D9FF1200E552E7CFD9FF1200640EF36E36
:10162000080ED7EF0BF00201D86B0201010ED26F4A
:10163000120005C0DBFF0A0E146E0E6E080EDBCF23
:1016400009F0FDEC15F0080E09C0DBFFC0EF0BF050
:10165000E96EEA6AD890E936EA36600EE926000EAD
:10166000EA221200FB0EDBCF14F0FC0EDBCF15F0EC
:10167000080EDB509C0F020D1450F324E96E155038
:10168000F4201200DFCFF6FF010EDBCFF7FF020ED2
:10169000DBCFF8FF1200080E156ADB34FE0B15369F
:1016A000146EFD0EDB501424E96EFE0EDB50152087
:1016B0001200D76F0201010ED86F0201D26F120023
:1016C0000201D950010FD36FDACFD4F20201120018
:1016D000EA6E090EDBCFEEFF0A0EDBCFEDFF120044
:1016E000E86BE96BE66BE76BE06BE16B120048D8E7
:1016F000040EE7CFDBFF120043D8060EE7CFDBFF77
:101700001200FD0EDBCFD3F2FE0EDBCFD4F21200BF
:10171000000EF722F8220800F550E66E12000001D4
:101720001624146E000E1720156E1200CD90CF6A8D
:10173000CE6ACD801200F36E080EF3CFDBFF1200ED
:10174000F36E070EF3CFDBFF1200FD0EDBCFE9FFD8
:10175000FE0EDBCFEAFF1200020DD950F324E96E32
:10176000DA50F420EA6E1200020143DF0001E85172
:10177000EE26E951ED22120048DFE652DF6A120040
:10178000DB50300FE76E1200E7CFDBFF0A0E34DFCD
:1017900005C0DBFF120002012CDFEE2A000EEF2253
:1017A0001200CFC2D7F23FDFDF6E00011200DBCFA5
:1017B000F4FFF350F45C1200010EECDEEF50120067
:1017C000E9DEE552E750120075DAF2A4FED7BDDA81
:1017D00003E02A0EBB6E01D0BB6A71D255DBDF502D
:1017E00000080AE2FE0EDBAE03D0010EE66E01D069
:1017F000E66AEADF95DAF3D7E55261D25BDAE652C0
:10180000080EDF6EDF50000811E2FE0EDBAE06D0E0
:10181000010EE66ED9DFE552E66A05D0E66AD4DF4E
:10182000E552010EE66ED0DF7BDAECD7E55247D207
:1018300041DA9492530ECB6EC40ED56E590ED66E0D
:10184000F2942A0EBB6E070EE66EF80EC2DA080E90
:10185000E66E950EBEDA040EE66E300EBADAFE0EB5
:10186000DBCFE6FFCBDFE552FD0EDBCFE6FFC6DFC9
:10187000E552E66AA9DFE552948221D21BDAF2A48E
:10188000FED763DA03E02A0EBB6E01D0BB6A17D223
:10189000FBDADF50000811E2FE0EDBAE06D0E66A8E
:1018A000EDDFE552010EE66E05D0010EE66EE6DFD5
:1018B000E552E66AE3DF34DAECD7E55200D2FAD932
:1018C0009492530ECB6EC50ED56EFA0ED66EF29470
:1018D000BB6A030EE66EC00EE66EDADFE552E55235
:1018E000FE0EDB50080DFE0EF3CFDBFF050EE66E9D
:1018F000FE0E80DAFD0EDB50040DFD0EF3CFDBFF94
:10190000060EE66EFD0E76DAE66AB8DFE5529482E0
:10191000D6D1D0D9130EE126FC0EDBCFF6FFFD0E9B
:10192000DBCFF7FFFE0EDBCFF8FF0900030ED1DAA5
:10193000040EF5CFDBFF010EC8DA0D0ECADA0E0E6B
:10194000F5CFDBFFBADAED1001E0ADD0020EE76EA5
:1019500057DAE7501626000E1722186AD890163666
:1019600017361836BADA1624F36EEE501720F46ED6
:10197000EE501820BADAF5CF14F00800F5CF15F0C4
:10198000830E1502F3CF15F01402F3CF14F0F450C8
:101990001526090EF3CFDBFF0A0E15C0DBFFB50ECF
:1019A000146E156A77DA33DA090EDBCF14F00A0EFB
:1019B00005DA70DA0B0E08C0DBFF0C0E09C0DBFF86
:1019C000BB6A030EE76E47D9050E83DA060EF5CF24
:1019D000DBFF040E7ADA070E7CDA080EF5CFDBFFA8
:1019E00094929EA2FED79E920B0EDB50BB6E030E0E
:1019F000DBCF14F0040EDBCF15F0050E1424DF6EE0
:101A000062D932DAAFD915E238D941D909E29EA2BA
:101A1000FED7010EDB06020E01E2DB069E92F5D731
:101A2000BB5004E10B0EDB50BB6E01D0BB6ADF2A5A
:101A3000E7D7E6D919DAB0EC15F016500624146E83
:101A400017500720156E050E1424DF6E3CD9070EC3
:101A5000DBCF1BF0080EDBCF1CF0050EDB501B2488
:101A6000196E060EDB501C201A6EC0D919C00DF07D
:101A70001AC00EF077D915E200D909D909E29EA261
:101A8000FED7010EDB06020E01E2DB069E92F5D7C1
:101A9000BB5004E10B0EDB50BB6E01D0BB6ADF2AEA
:101AA000D5D7948211D009DA06E1600EED1803E172
:101AB000C4D9BEDE07D001DA07E1500EED1804E10B
:101AC000BCD9FDDEE552E552130EE15C02E2E16AAB
:101AD000E552E16EF4D0EED8110EE126E1D90B0EFD
:101AE000EECFDBFF0C0EEDCFDBFFEBD9ED1001E00D
:101AF0009AD0020EBBD8EECF14F0EFCF15F0830EC4
:101B00001502F3CF15F01402F4501526070EF3CF8B
:101B1000DBFF080E15C0DBFFB50E146E156AC7D9C2
:101B2000070E08C0DBFF080E09C0DBFF070EDBCF86
:101B300014F0080E43D9BBD96AD9BB6A040E96D8F3
:101B4000030EEECFDBFF040EEDCFDBFF060E8ED8CB
:101B5000050EEECFDBFF060EEDCFDBFF94929EA2CB
:101B6000FED79E92090EDB50BB6E86D9B0EC15F005
:101B700007C015F0040E0624DF6EDFCF14F07CD909
:101B8000B1D81BE2640EDF5C02E2F9D801D0B9D80B
:101B900025D97DD809E29EA2FED7010EDB06020EF2
:101BA00001E2DB069E92F5D7BB5004E1090EDB5043
:101BB000BB6E01D0BB6ADF2AE0D7040EDF6EDFCF39
:101BC00014F0050EDBCF19F0060EDBCF1AF0030E72
:101BD000DB501924176E040EDB501A20186E06D93C
:101BE00017C00DF018C00EF07DD81BE2640EDF5C4C
:101BF00002E2C5D801D085D8F1D849D809E29EA221
:101C0000FED7010EDB06020E01E2DB069E92F5D73F
:101C1000BB5004E1090EDB50BB6E01D0BB6ADF2A6A
:101C2000CED7948211D04DD906E1600EED1803E1B4
:101C30000FD9FEDD07D045D907E1500EED1804E1BC
:101C400007D93DDEE552E552110EE15C02E2E16AA0
:101C5000E552E16E34D0DBCF14F0040EDBCF15F08B
:101C6000E7501426000E15220EEF0FF0E76E18D97C
:101C7000E750E926000EEA221200DFCF14F0156AC1
:101C8000CDD8010E26D9020EF5CFDBFF1200D950B8
:101C9000010FE96EDACFEAFF000ED880EE54000E95
:101CA000ED541200DBCF09F014C00DF015C00EF09A
:101CB000E7EF15F0D9CFE6FFE1CFD9FF1200E552EB
:101CC000E7CFD9FF1200DFCF14F0050EE76E030E49
:101CD000DBCF17F0040EDBCF18F0E7501726000E0D
:101CE00018221200B0EC15F006C015F007C016F06F
:101CF000040E1526000E16221550145C000E165404
:101D00001200FB0EDBCF14F0FC0EDBCF15F0640EDF
:101D1000DF5C020D1450F324E96E1550F42012001C
:101D2000E552FE0EDB50020DFE0EF3CFDBFFDF06A9
:101D30001200110ECED8120EF5CFDBFF110EDBCF45
:101D4000E6FF0F0EDBCFE6FF1200D650146E156AC9
:101D5000A60E145E000E155A1450D66EF294FE0EA6
:101D6000DB501200B0EC15F017500624156E185019
:101D70000720166E1550145C000E16541200156ADA
:101D8000DF34FE0B1536146EFD0EDB501424E96EA5
:101D9000FE0EDB50152012000F0EEECFDBFF100EF3
:101DA000EDCFDBFF0F0EDBCFE6FF0D0EDBCFE6FF47
:101DB0001200E96EDACFEAFFEE501200DBCF15F029
:101DC0001406000E155A1450CB6E020E146E156ACE
:101DD0001200E66E03DDE552E5521200EA6E010ED6
:101DE000EECFDBFF020EEDCFDBFF1200020E086E1E
:101DF000096A1200DBCFE6FF4BDDE552E552120027
:101E0000030EDBCF16F0040EDBCF17F01200090E25
:101E100008C0DBFF0A0E09C0DBFF1200166AD8906B
:101E200014361536163659D81424F36EEE50152094
:101E3000F46EEE50162075EF0FF0050E46D80F0E1B
:101E400048D8100EF5CFDBFF060E3FD899EF0EF005
:101E5000080E0CDF0D0EEECFDBFF0E0EEDCFDBFF1D
:101E60000A0E04DFCCEF0EF0C1DF050EDBCF0DF064
:101E7000060EDBCF0EF01200B9DF030EDBCF0DF044
:101E8000040EDBCF0EF0120015DFE652FD0EDB5024
:101E9000DF6E1200090EDBCF08F00A0E52EF0EF0D3
:101EA000FD0EDBCFE9FFFE0EDBCFEAFF1200070ECF
:101EB000DBCF08F0080E52EF0EF0D9500D0FD9EF1E
:101EC0000EF0D9500B0FD9EF0EF0E76E030E2BEF8B
:101ED0000EF0F5CFDBFF0A001200D950FC0FE96EBF
:101EE000FF0EDA20EA6EEE501200F86EF4CFF7FF24
:101EF000F3CFF6FF09001200040120511F0B010867
:101F000001E012002051600BE842E842E842E8425A
:101F1000E842010801E01200245103E0240501E039
:101F200012002151230A39E0010A33E0030A25E0B7
:101F3000010A1CE0240A31E0070A2FE0010A2DE023
:101F4000030A0EE0010A01E012004ED90201E40E7C
:101F5000F86F020EF96F0001FA930201080E17D014
:101F600043D90201E40EFA6F020E05D03DD90201F9
:101F7000D90EFA6F020EFB6F120036D90201D90E8C
:101F8000F86F020EF96F0001FA930201070EFC6F61
:101F900012002AD922C4E0F2120012000201D96B09
:101FA000C20EDA6F010EDB6FDC6BDD6BDE6B080ED1
:101FB000DF6FD26BD16B1A0E726E1E0E736E040140
:101FC000000E166F050E176F400E146F0401196F87
:101FD000080E1A6F050E1B6F880E186F0401480E4D
:101FE0001E6F050E1F6F400E1C6F1200D9CFE6FF4B
:101FF000E1CFD9FF0201D16B040118BF30D0FC0E34
:10200000DBCF14F01951D880145403E2FC0E19C42C
:10201000DBFF0201D16BFC0EDB50D15D19E2D15127
:10202000EA6A080FE96E050EEA22EF50E66ED1511A
:10203000E76EFD0EDBCFE9FFFE0EDBCFEAFFE750D8
:10204000E926000EEA22E552E750EF6ED12BE3D7E6
:102050000401400E196F1817187D880E181302011D
:10206000D151E552E7CFD9FF1200ACD80201D251CD
:1020700014E1DF6AB2D802E115500BE0FD0EDBCFB0
:10208000E9FFDB2AFE0EDBCFEAFF01E3DB2AEF509C
:10209000F1E175D8D86B010ED26F9AD093D80201B6
:1020A000D25115E1DF6A99D802E115500CE0FD0E1E
:1020B000DBCFF6FFDB2AFE0EDBCFF7FF01E3DB2AE7
:1020C0000800F550F0E15BD8010ED86FD26F80D0D8
:1020D00079D804011CBF52D0030E0201D25D01E188
:1020E000D26BD2514BE0020ED25D03E104011D6BB5
:1020F0003CD0D2053DE1400E146E156AD751145CF8
:10210000000E155803E2400EDF6E02D0D7C2DFFF8B
:10211000DFCF1DF4DF50D75DD76F480ED56F050EAA
:10212000D66FD8050AE1DF5011E0D3C2F6FFD4C262
:10213000F7FF0800F5503AD8F6D7DF5007E0D3C2D2
:10214000E9FFD4C2EAFFEF5031D8F7D70201D751E7
:102150000FE104011D51146E156A400E141805E1BB
:10216000155003E10201020E02D00201030ED26FEC
:10217000400E04011C171C7D880E1C1329D0DF5053
:10218000146E156AD950FD0FE96EFF0EDA20EA6E63
:102190001450EE5E1550ED5AFD0EDBCFD3F2FE0E5D
:1021A000DBCFD4F2DFCFD7F202011200D5C2E9FFB4
:1021B000D6C2EAFFEF6ED52B000ED623D32BD42345
:1021C000DF061200D9CFE6FFE1CFD9FFE6521200B9
:1021D000E552E552E7CFD9FF1200DF2ADF50146E37
:1021E000156AFF0E141812000201030EF76F120099
:1021F0006C5002E0000E01D0010E00090BE004015A
:1022000000513C0BE842E8420D0802E113EF11F0E7
:1022100045EF11F06C5002E0000E01D0010E0409F0
:1022200001E042D81200D9CFE6FFE1CFD9FFE65254
:102230000201F66BF76BFC6BFD6B47EC12F0DF6A8B
:10224000DF50146E156A010E145C000E15581AE268
:102250000201F75117E1F76ADF34FE0BF736F66E2D
:10226000BF0EF6262A0EF7220900F5CF14F008005B
:10227000F5CF15F004D015C0FAFF1450F96EFBDF4E
:10228000DF2ADED799D8E552F6D0020E0201F65DBC
:1022900009E168D8040100BD02D0C80E01D0880E43
:1022A000006F120015EF12F0040E0001F95D09E154
:1022B00022C46EFF6E50000802E2050E01D0030E2C
:1022C000F96F0201F60509E10AD8040104BD02D044
:1022D000C80E01D0880E046F120015EF12F0C4D89A
:1022E0000201080EFC5D000EFD5905E2FCC2DEFF96
:1022F000FDC2DDFF03D0080EDE6EDD6A040104932B
:102300000491010EDB500413DFCF05F4000EDB5007
:102310000201FC5F010EDB50FD5B280EFA6F040E1C
:10232000FB6F0001FAA30CD098D815E0F8C2F6FFB5
:10233000F9C2F7FF0800F55080D8F6E2DB06F4D7C3
:102340008CD809E0F8C2E9FFF9C2EAFFEF5075D86E
:10235000F7E2DB06F5D7020EE15C02E2E16AE55244
:10236000E16E89D081D8030E04010015E76E010EDD
:10237000E7CFDBFF01C4DFFFDE500201FC27DD50A9
:10238000FD23280EF86F040EF96F67D80EE0F8C22F
:10239000E9FFF9C2EAFFEF50FAC2E9FFFBC2EAFF28
:1023A000EF6E6DD8F2E2DB06F0D7020EE15C02E2DE
:1023B000E16AE552E16E5FD00201F75105E145D8CF
:1023C000840E006F04011DD0040120AF1CD0020157
:1023D000FC510401265D0201FD510401275904E26C
:1023E00026C4FCF227C4FDF27ADF0201010EF66F6B
:1023F0002CD8800E006F0401280E066F040E076FA4
:10240000C80E046F10D00201020EF66F0401056BB6
:10241000C80E046F0401080E016F280E026F040E2F
:10242000036FC80E006F6D9812000201F66B0DD895
:10243000880E006F0401046B1200FAC2E9FFFBC2B0
:10244000EAFFEF6E02013FEF12F00401080E016F88
:10245000200E026F040E036F1200D9CFE9FFDACF0E
:10246000EAFFEE50ED101200D9CFE6FFE1CFD9FF21
:10247000020EE1261200E552E7CFD9FF1200FA2B37
:10248000000EFB23F82BF923DF06010E12000401D6
:102490002051600BE842E842E842E842E842000985
:1024A00001E012002151070A40E00B0A3EE0070A52
:1024B00033E0010A23E00B0A1FE0020A1DE0030AD1
:1024C00019E0080A10E0010A0CE00F0A08E0030A0C
:1024D00001E0120012D90001040EF96F120096EF0C
:1024E00012F0CDEF12F009D90201FB0EF86F000EC9
:1024F000F96F0CD0E8EF12F01AEF13F002D90201D5
:10250000F86FF96BFC0EF827000EF9230001FA931F
:102510000201010EFC6F1200F4D8EA6AFC0FE96EAA
:10252000000EEA2222C4EFFF12001200800E040106
:10253000205D32E12351030A1FE0010A0AE0030A89
:1025400029E1DBD80201F40EF86F290EF96F120EA3
:102550001ED0ADD8B50EF6262A0EBBD8020E02014B
:10256000F76AF825F66EF951F7220900F5CFFCF26B
:102570000A00F5CFFDF20ED09AD8B90EF6262A0E33
:10258000A8D8F8C2F6FFF9C2F7FF0800F55002011B
:10259000FC6FFD6B0001FA831200AFD80F0EE66EE0
:1025A000710EE66E0F0E9DD8010EE66EFC0EE66E05
:1025B000000E97D822C4FBF00401225104E100016F
:1025C000050EF96F12000001060EF96FCEEF0FF045
:1025D0000401286B296B040120511F0B020A0FE034
:1025E000030A0BE0010A18E188D8040128810001E0
:1025F000FAA112D0040128830FD07FD80DD04BD878
:1026000001E0010E5DD8FAC2E9FFEA6EEF50040B5B
:1026100003E00401010E286F0201F7050AE102013F
:10262000280EF86F040EF96F0001FA930201020EF2
:10263000FC6F1200040122050EE120511F0B00095E
:102640000AE15BD8030E0401215D03E10001FA8178
:1026500002D00001FA91040122511CE120511F0B0C
:10266000020818E124510F0B000914E014D801E00E
:10267000010E26D8030E0401215D04E1840E38D832
:10268000EF6E120024AF03D033D8EF6A1200880E29
:102690002FD8EF6E120035D80F0B080DF350156AC6
:1026A000000F146E040E15222451800B120025D841
:1026B00004012251F66EF76AD890F636F73612000A
:1026C000040DF35002011424FA6F000E1520FB6F65
:1026D0001200F7220900F5CFF8F20A00F5CFF9F25F
:1026E0001200E66E2BEC14F0E552E552E5521200B2
:1026F000FAC2E9FFFBC2EAFF12000201010EF76F06
:102700001200FBDF0401245112006DA60CD8000159
:10271000F90508E16DBA06D0686A696A6980698856
:10272000020EF96F12006D6A696A6D860001010E72
:10273000F96F12006D6A696A0001F96B12009AEF75
:1027400013F00001F95101E112006850040B04E09C
:102750006950040B01E03CD86DB212006850010BC7
:1027600004E06950010B01E054D86850100B04E0FC
:102770006950100B01E024D86850400B04E0695008
:10278000400B01E03BD86850200B04E06950200B5F
:1027900001E036D86850020B04E06950020B01E0FA
:1027A00036D8030E0001F95D01E212006850080BF3
:1027B00006E06950080B03E0F8EC10F06896120090
:1027C000698468986D82A19AA08A0300A09A120079
:1027D0006D926994689412000001FAA10ED0F8DF9E
:1027E0006D840201080EFE6F070EFF6FFE07000EDC
:1027F000FF5BFE51FF11FAE16D941200689C12001C
:1028000070A003D015EC12F07090689A12006892D4
:1028100012006A6A686A9F0E6B6E7B0E696E6E6A42
:102820000F0EE66E710EE66E0F0EE66E14D8E552D0
:10283000E552E552160E706E68A602D06896FCD777
:102840006D9815EC12F00001FA910001FB6B00018C
:10285000030EF96F1200D9CFE6FFE1CFD9FFFD0ECD
:10286000DBCFE9FFFE0EDBCFEAFFFC0EDB5004E01E
:10287000EE6AFC0EDB06F9D7E552E7CFD9FF12006E
:10288000DACFE4FFE9CFE4FFEACFE4FFE6529EA40B
:102890005AD00001DDB121D0BD6A060EBD6E9E94F6
:1028A000DD81BF501E6E1D6ABE5000011D24EA6FFF
:1028B000000E1E20EB6F0001DE6BDF6B9EA009D0C7
:1028C0009E900001000ED880EA55010EEB5501E202
:1028D00082D80001E06BE16B41D09E94DD83BF5054
:1028E0001D6E1E6A1E6E1D6ABE5000011D24E66F1D
:1028F000000E1E20E76FDEC0E8F0DFC0E9F09EA00A
:1029000014D09E9068D80001E65D010EE75904E2FC
:102910000001E82B000EE9234CD807E353D804E369
:102920000001DD85F29C01D032D80001E02B000EC1
:10293000E1230001ED510001E05D0001EE510001D5
:10294000E1590CE306D09E9046D833D807E33AD835
:1029500004E30001DD85F29C01D019D8E552E5CFF2
:10296000EAFFE5CFE9FFE5CFDAFF1100D8CFE4FFBA
:10297000E0CFE4FFE46EDACFE4FFE652E552E5CFC4
:10298000DAFFE550E5CFE0FFE5CFD8FF100000010A
:10299000EC5126D8EECFE2F0EDCFE3F0EC29EC6F6E
:1029A000E8501ED8EECFE4F0EDCFE5F0EC29EC6F67
:1029B00012000001E2510001DE5D0001E35100015F
:1029C000DF5912000001E4510001E05D0001E55112
:1029D0000001E15912000001DE2B000EDF2312007E
:1029E000E96EEA6AD890E936EA36600EE926000E0A
:1029F000EA2212001201000202000008DB045B0060
:102A000000000102000109024300020100803209B6
:102A10000400000102020100052400100104240248
:102A200002052406000105240100010705820308B0
:102A3000000209040100020A000000070503024029
:102A40000000070583024000000403090434034822
:102A5000006F006D006500630069006E0065006D29
:102A60000061002D00660072002E0063006F006D93
:102A70000020002000200020002000200020002056
:102A800000340343006F006C006F00720069006D3A
:102A90000065007400720065002000480043004695
:102AA00000520020002000200020002000200020F4
:102AB0000020002000062A062A492A4D2A812AF8E9
:102AC0001EFF2A0EF66E080EF76E000EF86E02015B
:102AD0000900F550F16F0900F550F26F03E1F1675D
:102AE00001D03DD00900F550EC6F0900F550ED6FB5
:102AF0000900F550EE6F09000900F550E96E090074
:102B0000F550EA6E090009000900F550EF6F090061
:102B1000F550F06F09000900F6CFF3F2F7CFF4F2A9
:102B2000F8CFF5F2ECC2F6FFEDC2F7FFEEC2F8FF08
:102B30000201EF5302E1F05307E00900F550EE6E99
:102B4000EF07F8E2F007F9D7F3C2F6FFF4C2F7FF98
:102B5000F5C2F8FF0201F107000EF25BBFD71200C9
:102B600008C012F008500D02F4CF07F0F3CF06F0C2
:102B700009500E02F4CF09F0F3CF08F00D02F35024
:102B80000726F4500822E86A092212500E02F35078
:102B90000726F4500822E86A0922000C04D80FD84E
:102BA0002BEC04F0FCD70F0EC112140E6F6E000157
:102BB000F96B0001FA6B0001FB6B1CEF04F085EC74
:102BC00013F06FBE02D0A1EC13F068EF10F0056AAD
:102BD000046A100EE76ED8900836093604360536BA
:102BE0000D50045C0E50055805E30D50045E0E5068
:102BF000055A082AE72EF0D71200056A080EE76E7C
:102C0000D890093605360E50055C02E3056E092A98
:102C1000E72EF7D7120013EE00F023EE00F0F86A6B
:102C2000019C61EC15F0CEEC15F0FDD712000D0003
:102C300076352E33300D0A000D0A00303132303037
:102C40003400FCFF5C008000B70010006E0108003B
:102C50003803040001050000FE7F2E0040005C00E8
:102C60000800B70004009C01020080020000FF3F42
:102C7000170020002E0004005C000200CE000200BD
:102C800040010000FF3F170020002E0004005C0000
:102C90000200CE00020040010000FF1F0C001000E7
:102CA000170002002E00020067000200A0000000D2
:102CB000909192939495969798999A9B9C9DFFFFDB
:102CC000FFFFFFFFFFFFFFFFFFFFFFFFFFFFFFFF14
:102CD000FFFFFFFFFFFFFFFFFFFFFFFFFFFFFFFF04
:102CE000FFFFFFFFFFFFFFFFFFFFFFFFFFFFFFFFF4
:102CF000FFFFFFFFFFFFFFFFFFFFFFFFFFFFFFFFE4
:020000040020DA
:08000000010002FFFFFFFFFFFA
:020000040030CA
:0E000000200E391E008180000FC00FA00F409F
:0200000400F00A
:10000000FF00FF00FF00FF00FF00FF00FF00FF00F8
:10001000FF00FF00FF00FF00FF00FF00FF00FF00E8
:10002000FF00FF00FF00FF00FF00FF00FF00FF00D8
:10003000FF00FF00FF00FF00FF00FF00FF00FF00C8
:10004000FF00FF00FF00FF00FF00FF00FF00FF00B8
:10005000FF00FF00FF00FF00FF00FF00FF00FF00A8
:10006000FF00FF00FF00FF00FF00FF00FF00FF0098
:10007000FF00FF00FF00FF00FF00FF00FF00FF0088
:10008000FF00FF00FF00FF00FF00FF00FF00FF0078
:10009000FF00FF00FF00FF00FF00FF00FF00FF0068
:1000A000FF00FF00FF00FF00FF00FF00FF00FF0058
:1000B000FF00FF00FF00FF00FF00FF00FF00FF0048
:1000C000FF00FF00FF00FF00FF00FF00FF00FF0038
:1000D000FF00FF00FF00FF00FF00FF00FF00FF0028
:1000E000FF00FF00FF00FF00FF00FF00FF00FF0018
:1000F000FF00FF00FF00FF00FF00FF00FF00FF0008
:10010000FF00FF00FF00FF00FF00FF00FF00FF00F7
:10011000FF00FF00FF00FF00FF00FF00FF00FF00E7
:10012000FF00FF00FF00FF00FF00FF00FF00FF00D7
:10013000FF00FF00FF00FF00FF00FF00FF00FF00C7
:10014000FF00FF00FF00FF00FF00FF00FF00FF00B7
:10015000FF00FF00FF00FF00FF00FF00FF00FF00A7
:10016000FF00FF00FF00FF00FF00FF00FF00FF0097
:10017000FF00FF00FF00FF00FF00FF00FF00FF0087
:10018000FF00FF00FF00FF00FF00FF00FF00FF0077
:10019000FF00FF00FF00FF00FF00FF00FF00FF0067
:1001A000FF00FF00FF00FF00FF00FF00FF00FF0057
:1001B000FF00FF00FF00FF00FF00FF00FF00FF0047
:1001C000FF00FF00FF00FF00FF00FF00FF00FF0037
:1001D000FF00FF00FF00FF00FF00FF00FF00FF0027
:1001E000FF00FF00FF00FF00FF00FF00FF00FF0017
:1001F000FF00FF00FF00FF00FF00FF00FF00FF0007
:00000001FF
